:100000000C9461020C94A5020C94A5020C94A50218
:100010000C94A5020C94A5020C94A5020C94A502C4
:100020000C94A5020C94A5020C9452140C94241563
:100030000C9486220C94A5020C94A5020C94A502A3
:100040000C94A5020C9407030C94A5020C94A50231
:100050000C94A5020C94EE220C94A5020C94A5021B
:100060000C94A5020C94A5020C94A5020C94A50274
:100070000C94A5020C94A5020C94A5020C94A50264
:100080000C94C70A0C94A5020C94A5020C94A5022A
:100090000C94A5020C94A5020C94A5020C94A50244
:1000A0000C94A5020C94A5020C94A5029115B3150D
:1000B000A116B315A116F8151B16A11670168316F6
:1000C0006D196D199C199C19DB19FB19511B511BDA
:1000D000061A511BB61AB61A1D1B261B511B4B1BA9
:1000E000C31AC31AC31AC31AC31AC31AC31AC31A28
:1000F000C31AC31AC31AC31AC31AC31AC31AC31A18
:10010000D31AE11AE81AEF1AF91A07634236B79BB5
:10011000D8A71A39685618AEBAAB558C1D3CB7CC67
:100120005763BD6DEDFD753EF6177231BF000000DF
:10013000803F08000000BE922449123EABAAAA2AC2
:10014000BECDCCCC4C3E00000080BEABAAAAAA3EDD
:1001500000000000BF000000803F00000000000819
:100160004178D3BB4387D1133D190E3CC3BD4282B6
:10017000AD2B3E68EC8276BED98FE1A93E4C80EF74
:10018000FFBE01C4FF7F3F00000000000000000030
:1001900000000000000000010204060A0F17202CD6
:1001A0003A4A5D71879DB3C7DAE9F5FCFFFCF5E9D2
:1001B000DAC7B39D87715D4A3A2C20170F0A0604EF
:1001C0000201000000000000000000002B001400ED
:1001D0001A000800150017001C0018000C0012007F
:1001E00013002A00290004001600070009000A0075
:1001F0000B000D000E000F003300015201001D0026
:100200001B00060019000500110010003600370021
:10021000380001000030E300E200E000E1002C00C3
:100220002C0002522D00340028000100010049007A
:100230004A0052004D004B000100400041004200C6
:100240004300010001004C00500051004F004E00DF
:1002500001003D003E003F0044000100010001009C
:10026000010001000100010001003A003B003C00D8
:100270004500010001000100010001000100010032
:100280000100AA00A900AB00AE00010001001E029F
:100290001F022F02300231024B00240025002600ED
:1002A000250201000100200221022602270235005A
:1002B0004E002100220023002E0201000100220234
:1002C00023022F003000350224021E001F002000F0
:1002D000310001000100010049000100010001009E
:1002E00001000100010027002E0001002803540036
:1002F00068006500200050006C0061006E00630023
:100300006B0020004B006500790062006F00610007
:100310007200640000002C034F007200740068003B
:100320006F006C0069006E006500610072002000C3
:100330004B006500790062006F006100720064008C
:10034000730000000403090409026D00040100A009
:10035000FA09040000010301010009211101000153
:10036000223F000705810308000A09040100010378
:10037000010200092111010001224D00070582033D
:1003800008000A090402000103000000092111010C
:1003900000012236000705830308000A0904030050
:1003A00001030000000921110100012239000705A5
:1003B00084031000011201100100000008EDFE602E
:1003C0006001000102000105010906A101050719EC
:1003D000E029E71500250195087501810205081936
:1003E0000129059505750191029501750391010596
:1003F000071900297715002501957875018102C03C
:1004000005010980A101850216010026B7001A0125
:10041000002AB700751095018100C0050C0901A1E3
:10042000018503160100269C021A01002A9C027510
:100430001095018100C005010902A1010901A10077
:100440000509190129051500250195057501810288
:100450009501750381010501093009311581257F59
:1004600095027508810609381581257F9501750863
:100470008106050C0A38021581257F9501750881D2
:1004800006C0C005010906A101050719E029E71505
:100490000025019508750181029501750881010506
:1004A00008190129059505750191029501750391BA
:1004B000010507190029FF150025FF95067508811C
:1004C00000C011241FBECFEFDAE0DEBFCDBF04B6FF
:1004D00003FE24C080911E0390911F03A09120036E
:1004E000B09121038730904BA740B04BB9F41092E4
:1004F0001E0310921F03109220031092210314BEBA
:1005000084B7877F84BF88E10FB6F894809360003A
:10051000109260000FBEE0E0F8E3099511E0A0E062
:10052000B1E0E6E6F9E502C005900D92A03CB10706
:10053000D9F713E0A0ECB1E001C01D92AE31B107D4
:10054000E1F70E9498110C94B12C0C9400000895CE
:10055000089581E0089508950C94A8020C94A902CE
:100560000C94AB020E947B2823E030E0281B310969
:10057000220F2093C4010895282F2F988091800086
:10058000211108C0877F8093800010928D00109207
:100590008C001BC0886080938000233019F48FEF9B
:1005A0009FEF0FC083E090E0821B9109880F991F95
:1005B0002FEF3FEFA90102C0569547958A95E2F7C4
:1005C000CA0190938D0080938C000C94B2020E941B
:1005D000B20284E08093C3011092C0010895279A6B
:1005E0002F988FEF9FEF90938700809386008AE08B
:1005F0008093800089E1809381000E94E4270C941D
:10060000E7020E94EF026E9A769A0C94A7021F925C
:100610000F920FB60F9211242F933F938F939F93B6
:10062000EF93FF93E091C101F091C201CF010196D8
:100630009093C2018093C1010090C30102C0F6955E
:10064000E7950A94E2F7EF738091C001823019F4C4
:10065000E03251F404C0813039F4EF3329F4809151
:100660006F008D7F80936F00F0E0E457FE4FE491C0
:1006700021E031E0E29FC001E39F900D1124009042
:10068000C40102C0969587950A94E2F790938D0075
:1006900080938C00FF91EF919F918F913F912F91CB
:1006A0000F900FBE0F901F90189561110DC0FC01A7
:1006B0008281882331F085EE0E9411180E943B2828
:1006C00003C085EE0E94D91880E090E0089581E093
:1006D00008950C94670308950C940103809115020A
:1006E000882309F448C08091D1019091D2010097EC
:1006F00079F40E94B8229093D2018093D101809125
:10070000D30190E0009771F48091D40190E00AC089
:100710000E94C4222091000130910101281739075D
:1007200040F329C00197880F991F880F991FFC017A
:10073000EB52FE4F60817181828193810E942D0A6C
:10074000E091D30184E0E89FF0011124EB52FE4FC9
:1007500060817181828193814FE050E00E94E50DBC
:100760008091D30190E001966091D40170E00E94E5
:10077000612C8093D3010C94AC02109217020C945C
:10078000FA090895089581E0809317020C94C2033A
:10079000089508958F929F92AF92BF92EF92FF9229
:1007A0000F931F93CF93DF93CDB7DEB7A3970FB609
:1007B000F894DEBF0FBECDBF7C01FC01008111812A
:1007C000C8010E94B520B8010E94CC058C01B70178
:1007D0000E946903882309F4CCC10032F0E51F07A9
:1007E00041F4F7018281882309F458C00E94490E20
:1007F000C0C10132F0E51F0741F4F701828188236F
:1008000009F44CC00E94520EB4C10232F0E51F0739
:1008100051F4F7018281882309F440C00E94450EFB
:100820008111F0CFE3CF0332F0E51F0739F4F70170
:100830008281882399F10E94C3039BC10432F0E5B1
:100840001F0739F4F7018281882341F10E94BD031B
:1008500090C10532F0E51F0749F4F7018281882332
:10086000E9F0809117028111F1CFE5CF0632F0E572
:100870001F0739F4F7018281882381F00E94590E05
:100880000AC00732F0E51F0749F4F7018281882387
:1008900029F00E94640E0E94C9036BC18091170267
:1008A000811105C0F70182818111CFC018C1003EBE
:1008B000110579F4F7018281882309F44DC00E9463
:1008C000FA0981E080931602109215021092D40169
:1008D00050C1023E110559F4F70182818823E1F1EC
:1008E0000E94FA09109216021092150242C1033EAC
:1008F000110591F4F7018281882371F10E94FA09B0
:100900001092160281E0809315021092D30110928A
:10091000D2011092D1012DC10235110559F4F70110
:100920008281882309F425C1809100019091010101
:100930000A970DC00135110579F4F70182818823EA
:1009400009F417C180910001909101010A969093DA
:100950000101809300010DC14091040183E2EFE1A8
:10096000F1E0DE01119601900D928A95E1F7F70111
:10097000808121E030E02C0F3D1F280F311DC9017F
:100980002091020130910301FC01E20FF31F60810D
:10099000772767FD7095640F711D882777FD809517
:1009A000982F0E94832920E030E040E451E40E9427
:1009B000E8284B015C01F701218184E090E0821B73
:1009C0009109BC01882777FD8095982F0E94832983
:1009D0009B01AC01C501B4010E9480289B01AC01C0
:1009E00060E070E080E090E40E94F62A20E030E0D1
:1009F0004CED50E40E94932A4B015C01F701828187
:100A00008823D1F04FE050E0C501B4010E94E50D0C
:100A1000809116028823A1F08091D40124E0829F66
:100A2000F0011124EB52FE4F80829182A282B382A8
:100A30008F5F8093D40104C0C501B4010E942D0AC8
:100A40000F3F110508F02ECF94C08091D001811185
:100A50001FC0043130E5130709F051C00E946B0339
:100A600081E08093D0010E94B8229093CF018093BF
:100A7000CE011092C7011092C9011092C8011092C4
:100A8000CB011092CA011092CD011092CC0171C01D
:100A90008091CE019091CF010E94C422883C9105A3
:100AA00070F48091C701E82FF0E0EE0FFF1FE853CC
:100AB000FE4F118300838F5F8093C7015AC00438B3
:100AC00080E5180721F00538104501F13AC0F7011B
:100AD0008281882341F01092C50182E01EC0043853
:100AE00030E5130759F58091C501811106C086E2F2
:100AF0000E94111886E20E94D91882E01CC00438B6
:100B0000F0E51F0741F305381045D9F4F70182815C
:100B1000882331F01092C60180E20E94281929C072
:100B20008091C601811106C087E20E94111887E2F8
:100B30000E94D91880E20E942F191BC00538104569
:100B400029F381E08093C5018093C601C701A39674
:100B50000FB6F894DEBF0FBECDBFDF91CF911F91CE
:100B60000F91FF90EF90BF90AF909F908F900C945B
:100B7000AE0280E0A3960FB6F894DEBF0FBECDBFE5
:100B8000DF91CF911F910F91FF90EF90BF90AF90A9
:100B90009F908F90089508959CE0799FF001112413
:100BA00090E3899FE00DF11D1124E60FF11DEE0F7A
:100BB000FF1FE453FE4F859194910895880F991F6C
:100BC000FC01E45BFF4F859194910895880F991F74
:100BD000FC01E453FE4F8591949108950F931F9368
:100BE000CF93DF93EC01811521E39207A0F5C115A6
:100BF00080E3D80708F0D7C0C83ED105D8F4C03E7E
:100C0000D10508F007C2C83AD10578F4C53AD10534
:100C100008F06AC0C130D10509F463C008F4F7C117
:100C2000C430D10508F0F6C1F2C1CB3BD10508F4C0
:100C300066C0EDC1C11590E2D90708F0AFC0C1157B
:100C400021E0D20708F0E6C1C03FD10508F4DFC1BA
:100C50008E0110651FC2C03880E5D80700F5C03787
:100C600090E5D90708F0A3C0C11520E5D20709F423
:100C7000ACC050F4CE01905480319F4008F0C7C101
:100C8000DF708E01106A06C2C13080E5D80709F412
:100C9000AEC0C43190E5D90708F4AFC0B8C1C338BD
:100CA00020E5D20709F48EC050F4C13890E5D90789
:100CB00009F482C008F083C000E011EDEBC1C0313F
:100CC00081E5D80708F4A3C1C11597E5D90708F451
:100CD00036C1CE0190578115904108F098C1DF7060
:100CE00093C101E010E0D6C1C53AD10509F494C121
:100CF000C63AD10509F093C102E810E4CBC1C83A65
:100D0000D10509F48FC1C93AD10509F48EC1CA3A97
:100D1000D10509F48DC1CB3AD10509F48CC1CC3A87
:100D2000D10509F48BC1CD3AD10509F48AC1C03B84
:100D3000D10509F489C1CE3AD10509F488C1CF3A69
:100D4000D10509F487C1C13BD10509F486C1C23B75
:100D5000D10509F485C1C33BD10509F484C1C43B65
:100D6000D10509F483C1C53BD10509F482C1C63B55
:100D7000D10509F481C1C73BD10509F480C1C83B45
:100D8000D10509F47FC1C93BD10509F47EC1CA3B35
:100D9000D10509F47DC100E014E47CC1CE019F704F
:100DA0000E94E60578C1DD278E01106C73C1CF70FB
:100DB000DD278E01146D6EC100E010ED6BC100E007
:100DC00012ED68C100E013ED65C10E94BC1B0E94DA
:100DD000FA090E94C1038FEF94E32CE08150904008
:100DE0002040E1F700C000000E94132353C180910E
:100DF000F20281608093F2024DC10E94742381113E
:100E000002C00E9450230E94872390E090931D030C
:100E100080931C03C23080E5D80721F480911C0325
:100E2000816086C0C43090E5D90721F480911C030D
:100E300082607EC0C63020E5D20721F480911C0379
:100E4000846076C0C83080E5D80719F480911C030F
:100E500027C0CA3090E5D90721F480911C03806136
:100E600067C0CC3020E5D20721F480911C0380625A
:100E70005FC0CE3080E5D80721F480911C038064E8
:100E800057C0C03190E5D90721F480911C038068D8
:100E90004FC0C23120E5D20729F480911C03846041
:100EA000886046C0C33080E5D80721F480911C03D8
:100EB0008E7F3EC0C53090E5D90721F480911C0398
:100EC0008D7F36C0C73020E5D20721F480911C0306
:100ED0008B7F2EC0C93080E5D80719F480911C03A0
:100EE00026C0CB3090E5D90721F480911C038F7E7A
:100EF0001FC0CD3020E5D20721F480911C038F7DE7
:100F000017C0CF3080E5D80721F480911C038F7B78
:100F10000FC0C13190E5D90721F480911C038F7770
:100F200007C0C331D04531F480911C038B7F877F8C
:100F300080931C0380911C030E948B23ABC08D2FD8
:100F400099278F70992781309105D9F49E012370DC
:100F5000332702C0880F991F2A95E2F79C688E01FB
:100F600044E0000F111F4A95E1F700271370802B12
:100F7000912B53E0CC0FDD1F5A95E1F7C076DD27AA
:100F80002FC08230910531F4DC2FCC278E01016F08
:100F9000106A80C08330910569F4CE01837099276F
:100FA00001E010E002C0000F111F8A95E2F7C801AE
:100FB0009C680FC084309105B9F4CE0183709927E5
:100FC00001E010E002C0000F111F8A95E2F7C8018E
:100FD0009A6823E0CC0FDD1F2A95E1F7C07ED77019
:100FE0008C010C2B1D2B56C08530910531F4DC2F64
:100FF000CC278E01046F106A4DC0069709F04AC0D5
:10100000CF71DD27DC2FCC278E01106243C000E0BA
:1010100010E040C08E013EC001E810E43BC003E890
:1010200010E438C002EE14E435C009EE14E432C016
:101030000AEE14E42FC005EB14E42CC006EB14E414
:1010400029C007EB14E426C00CEC14E423C00DEC1B
:1010500014E420C003E815E41DC00AE815E41AC032
:1010600002E915E417C004E915E414C001E216E42E
:1010700011C003E216E40EC004E216E40BC005E260
:1010800016E408C006E216E405C007E216E402C052
:101090000AE216E4C801DF91CF911F910F910895E4
:1010A0009CE0799FF001112490E3899FE00DF11DF0
:1010B0001124E60FF11DEE0FFF1FE453FE4F859143
:1010C0009491803E9105E0F4803C910558F5813380
:1010D000910509F46FC048F48932910509F463C0A1
:1010E0008A32910509F46DC072C089339105E9F027
:1010F00082389105D1F08533910509F44DC067C060
:10110000833E910581F138F4803E9105B9F0823E2D
:101110009105D9F05CC0863E910561F1873E91054D
:10112000A1F155C00E94DE05089520911C0320FD09
:1011300002C021FF4CC080EE90E049C080911C03AA
:1011400080FFF9CF89E390E042C080911C0382FFC9
:101150000EC080911C0384FF03C080E090E037C084
:1011600083EE90E034C080911C0382FFF2CF82EEC8
:1011700090E02DC080911C0383FF0BC080911C0365
:1011800084FDEBCF87EE90E022C080911C0383FFAB
:10119000F5CF86EE90E01BC080911C0385FF07C051
:1011A00089E290E014C080911C0385FFF9CF85E3AC
:1011B00090E00DC080911C0386FF07C08AE290E09A
:1011C00006C080911C0386FFF9CF81E390E00E9466
:1011D000EE0508950C94B002E82FF0E0E25BFE4FBC
:1011E0008081E82FEF70F0E082958F7021E030E091
:1011F000A90102C0440F551F8A95E2F740A3089544
:101200000F931F93CF93DF9385B7806885BF85B712
:10121000806885BFC3E0D0E001E010E0FE01E25B42
:10122000FE4F8081E82FEF70F0E021A182958F7052
:10123000A80102C0440F551F8A95E2F7CA01822B0C
:1012400081A38C2F0E94EC08219740F78BE090E05F
:1012500061E070E0FC01EE5BFE4F2081E22FEF7059
:10126000F0E042A122952F70DB0102C0AA0FBB1F44
:101270002A95E2F79D01242B22A3019758F7DF91CD
:10128000CF911F910F910C946C03EF92FF920F93EB
:101290001F93CF93DF9300E212E0C3E0EE24E394C8
:1012A000F12CD5E08C2F0E94EC088BE090E040E020
:1012B00050E0FC01EE5BFE4F6081E62FEF70F0E046
:1012C00020A130E062956F7002C0359527956A9530
:1012D000E2F720FD09C09701082E02C0220F331F3C
:1012E0000A94E2F7422B532B019718F7F8019291D9
:1012F00082918F018417950721F051834083D09309
:1013000005018C2F0E94EC08C15060F68091050108
:1013100087FD2CC08150809305018F3F39F08FE904
:101320009FE00197F1F700C0000020C080911E02ED
:1013300090911F02909327028093260280911C02B5
:1013400090911D02909325028093240280911A02AD
:1013500090911B02909323028093220280911802A5
:101360009091190290932102809320020E946E03B3
:1013700081E0DF91CF911F910F91FF90EF90089541
:10138000E82FF0E0EE0FFF1FE05EFD4F80819181BE
:10139000089508950F931F93CF9308E212E0C0E0E1
:1013A000F801929182918F010E943022C80FF2E0E1
:1013B00000321F07A9F78C2FCF911F910F9108952D
:1013C0000E947423811102C00E9450230E9499231D
:1013D000809307033E9A809171008D7F8093710006
:1013E00082E0809390008AE18093910081E0809375
:1013F0002A02089580912A02811102C00E94E00908
:1014000010927A0210927902809171008D7F809300
:101410007100809190008F738093900010923C0235
:1014200010923B0210927302109274021092750295
:10143000109276021092720210927102E1E5F2E0CF
:10144000A1E4B2E011921192119211921D921D929B
:1014500082E0E137F807B1F70895CF92DF92EF927B
:10146000FF920F931F93CF93DF9320913B02222390
:1014700009F484C06B017C0180912A02811102C0B1
:101480000E94E00901E712E0C7E0D0E0A701960161
:10149000F80192918291729162918F010E94E428E9
:1014A000811131C0FE01EE0FFF1FEE0FFF1FEF5A3B
:1014B000FD4F1082118212821382DE01AA0FBB1F20
:1014C000AF5BBD4F11961C921E92C730D105E9F05B
:1014D000219644815581668177814083518362835F
:1014E0007383148215821682178212968D919C91B5
:1014F000139711969C938E9313961C921E9212979B
:1015000034961296E2CF219708F680917902909155
:101510007A02019797FD05C090937A028093790231
:1015200004C010927A02109279028091790290910F
:101530007A0220917702309178022817390724F037
:101540001092780210927702892BC1F48091710079
:101550008D7F80937100809190008F7380939000B5
:101560001092730210927402109275021092760219
:10157000109272021092710210923B02DF91CF9191
:101580001F910F91FF90EF90DF90CF9008951F92E1
:101590000F920FB60F9211244F925F926F927F922B
:1015A0008F929F92AF92BF92CF92DF92EF92FF9273
:1015B0002F933F934F935F936F937F938F939F935B
:1015C000AF93BF93CF93DF93EF93FF9380913B0251
:1015D000882309F49BC1C0917902D0917A021C162C
:1015E0001D060CF093C140902B0250902C0260908D
:1015F0002D0270902E0220E030E0A901C301B2015B
:101600000E948F2A18160CF065C0C130D10509F46C
:1016100052C08091770290917802BE010E94612CA5
:101620007C01909378028093770280903D029090A5
:101630003E02A0903F02B090400220E030E040E83F
:101640005FE3C501B4010E94802860933D0270935E
:101650003E0280933F0290934002F701EE0FFF1F7E
:10166000EE0FFF1FEF5AFD4FA301920160817181C0
:10167000828193810E94E82820E030E040E05EE330
:101680000E94932A9B01AC01C501B4010E948F2ADC
:1016900018168CF4C7010196BE010E94612C90932C
:1016A00078028093770210923D0210923E021092CF
:1016B0003F0210924002E0917702F0917802EE0F23
:1016C000FF1FEE0FFF1FEF5AFD4F60817181828176
:1016D0009381D0C0C0907302D0907402E0907502E4
:1016E000F090760220E030E0A901C701B6010E9427
:1016F000E4282197882309F4A2C0FE01EE0FFF1F02
:10170000EE0FFF1FEF5AFD4F80809180A280B380C3
:10171000A5019401C701B6010E94E42887FF31C0EA
:10172000A501940160E070E08CED93EC0E94E82844
:1017300020E030E040E451E40E94E82820E030E07E
:1017400040E05FE30E94932A9B01AC0160E070E0FF
:1017500080E090E40E94F62A9B01AC01C501B4012F
:101760000E94932A9B01AC01C701B6010E94E428A4
:1017700087FF07C0A701960160E070E08CED93E45D
:1017800039C0A5019401C701B6010E948F2A18161D
:101790000CF055C0A501940160E070E08CED93E47D
:1017A0000E94E82820E030E040E451E40E94E8286C
:1017B00020E030E040E05FE30E94932A9B01AC010F
:1017C00060E070E080E090E40E94F62A9B01AC01AA
:1017D000C501B4010E94932A9B01AC01C701B60167
:1017E0000E948F2A18165CF5A701960160E070E050
:1017F0008CED93EC0E94E82820E030E040E451E4D6
:101800000E94E82820E030E040E05FE30E94932A55
:101810009B01AC0160E070E080E090E40E94F62A59
:101820009B01AC01C701B6010E94932A6093730229
:1018300070937402809375029093760213C0FE0138
:10184000EE0FFF1FEE0FFF1FEF5AFD4F80819181BA
:10185000A281B3818093730290937402A093750266
:10186000B093760260917302709174028091750258
:101870009091760220912802309129022F3F4FEF5C
:10188000340731F02F5F3F4F309329022093280215
:101890000E946F0E6B017C0120E034E244EF51E4C2
:1018A0000E94E42887FF08C086EFC82E88E2D82E61
:1018B00084EFE82E81E4F82E20E030E040E051E4AF
:1018C000C701B6010E94932A9B01AC0160E074E25B
:1018D00084E79BE40E94E8286B017C010E94552963
:1018E0007093970060939600209106013091070154
:1018F0004091080150910901C701B6010E94932A45
:101900000E945529709399006093980080913C0241
:10191000882309F433C1C0903702D0903802E09098
:101920003902F0903A0220E030E0A901C701B60187
:101930000E948F2A1816D4F58091280290912902CE
:101940008F3F2FEF920729F0019690932902809301
:101950002802C701B6010E946F0E20E030E040E08F
:1019600051E40E94932A9B01AC0160E074E284E799
:101970009BE40E94E8286B017C010E94552970932A
:1019800097006093960020910601309107014091E5
:10199000080150910901C701B6010E94932A0E94D3
:1019A0005529709399006093980008C01092970091
:1019B0001092960010929900109298006091310256
:1019C000709132026F5F7F4F7093320260933102E9
:1019D000209196003091970080E090E0232BF1F069
:1019E000C0919600D09197000E9481296B017C01E3
:1019F000BE0180E090E00E9481299B01AC016091D2
:101A000033027091340280913502909136020E9427
:101A1000E82820E03FEF4FE757E410C00E948129FB
:101A20006B017C0120E030EE4FEF54E46091330213
:101A30007091340280913502909136020E94932A6F
:101A40009B01AC01C701B6010E948F2A87FD96C099
:101A500080912F028F5F80932F0290E020910303EB
:101A60003091040382179307A0F080910E0388231E
:101A700019F010922F020DC0809171008D7F80931C
:101A80007100809190008F738093900010923C02BF
:101A90007DC080913002C0912F02811128C0C0907A
:101AA0000803D0900903E0900A03F0900B0320E0B4
:101AB00030E0A901C701B6010E948F2A1816BCF4B4
:101AC00081E0809330021092370210923802109217
:101AD000390210923A02C0923302D0923402E0925C
:101AE0003502F0923602C150C0932F0243C01092CB
:101AF00030021092290210922802E0910503F09121
:101B0000060348E0C49FE00DF11D112480819181FE
:101B1000A281B3818093370290933802A093390257
:101B2000B0933A0220E030E040E85EE364817581E2
:101B3000868197810E94932A6B017C0180910A0122
:101B4000682F70E080E090E00E94812920E030E082
:101B500048EC52E40E94E8289B01AC01C701B601A1
:101B60000E94932A6093330270933402809335026B
:101B70009093360210923202109231028091070344
:101B800080FD04C010923C0210923B02FF91EF9145
:101B9000DF91CF91BF91AF919F918F917F916F9185
:101BA0005F914F913F912F91FF90EF90DF90CF90F9
:101BB000BF90AF909F908F907F906F905F904F906D
:101BC0000F900FBE0F901F901895CF92DF92EF925B
:101BD000FF92CF93DF936B017C01EA0180912A028F
:101BE000811102C00E94E0098091070380FF46C076
:101BF0008091790290917A0208970CF03FC0809111
:101C000071008D7F8093710080913C0281110E9450
:101C1000FA0981E080933B02109229021092280277
:101C200020E030E0A901C701B6010E948F2A1816F2
:101C3000DCF48091790290917A02FC01EE0FFF1F93
:101C4000EE0FFF1FEF5AFD4FC082D182E282F38276
:101C5000FC01EE0FFF1FEF5BFD4FD183C0830196A8
:101C600090937A02809379028091710082608093D0
:101C7000710080919000806880939000DF91CF91F7
:101C8000FF90EF90DF90CF900895809107038170CF
:101C90000895809107038160809307030E949D232C
:101CA0000C94C803809107038E7F809307030C94E4
:101CB0009D2380917B0290E0019666E070E00E9497
:101CC000612C80937B02089580917B0290E00197C4
:101CD00066E070E00E94612C80937B0208958F92F1
:101CE0009F92AF92BF92CF92DF92EF92FF920F93AB
:101CF0001F93CF93DF936B017C01C0912802D09199
:101D00002902BE0180E090E00E9481294B015C0124
:101D1000A701960160E070E08CE594E40E94E82859
:101D20009B01AC01C501B4010E94932A0E94552970
:101D300020917B02233009F473C028F4222351F050
:101D40002130E9F02CC1243009F4A0C0253009F479
:101D5000E0C025C180E090E0A0E0BFE380930601F1
:101D600090930701A0930801B093090110922B02F0
:101D700010922C0210922D0210922E0210C110927D
:101D80002B0210922C0210922D0210922E0264311E
:101D9000710540F46A30710560F520E030E040E8FC
:101DA0005EE32BC0693C710508F0AAC080E090E0BA
:101DB0000E94812920E030E040EA51E40E947F281F
:101DC00020E030E044E353E40E94E8289B01AC01AA
:101DD0000E94932A20E030E040E05EE30E94932AD4
:101DE0009B01AC0160E070E080E09EE30E947F28F0
:101DF00044C020E030E040E05FE3C701B6010E944C
:101E0000932A6B017C0180E090E0A0E0BEE3809328
:101E1000060190930701A0930801B0930901BFC088
:101E200010922B0210922C0210922D0210922E0270
:101E30004AE0469F9001479F300D1124C90168EB8D
:101E40007BE00E944D2CBC016C5D754077FF03C0A8
:101E5000719561957109882777FD8095982F0E946B
:101E600083292EE333EC4EE259E30E94932A20E0CB
:101E700030E040EC5EE30E9480286093060170939E
:101E80000701809308019093090189C010922B02E9
:101E900010922C0210922D0210922E02CE0183700D
:101EA0009927892BE1F0BE016170772780E090E0EF
:101EB0000E94812920E030E040E05EE30E94932A06
:101EC00020E030E040E45FE30E9480286093060158
:101ED0007093070180930801909309010CC080E082
:101EE00090E0A0E0BFE38093060190930701A093E8
:101EF0000801B0930901C770DD27CD2B09F04FC051
:101F00001092060110920701109208011092090127
:101F100046C010922B0210922C0210922D021092A9
:101F20002E0200E010E020E03FE300930601109352
:101F3000070120930801309309016739710578F191
:101F400080E090E00E94812920E030E047E153E406
:101F50000E947F2820E030E04AE754E40E94E8280D
:101F600020E030E048E452E40E94932A20E030E090
:101F700040EA51E40E94C5290E945029660F771F4C
:101F8000660F771FFB01EE5AFE4F2081318142819F
:101F90005381C701B6010E94932A6B017C01C701DE
:101FA000B601DF91CF911F910F91FF90EF90DF90DD
:101FB000CF90BF90AF909F908F90089580918C02AA
:101FC0000895CF93DF9300D01F92CDB7DEB79C0169
:101FD00080911303843019F593E099833B832A831E
:101FE0009093E9008FEF9091E800815095FD06C035
:101FF00095ED9A95F1F700008111F5CF8091E800F9
:1020000085FF0DC040E050E063E070E0CE01019636
:102010000E9442128091E8008E778093E8000F9032
:102020000F900F90DF91CF910895CF93DF9300D061
:102030001F92CDB7DEB720911303243021F522E0A3
:1020400029839B838A8383E08093E9008FEF9091BB
:10205000E800815095FD06C095ED9A95F1F70000D6
:102060008111F5CF8091E80085FF0DC040E050E080
:1020700063E070E0CE0101960E9442128091E80078
:102080008E778093E8000F900F900F90DF91CF91A3
:102090000895209113032430F1F422E02093E90005
:1020A0002FEF3091E800215035FD06C035ED3A950F
:1020B000F1F700002111F5CF2091E80025FF0BC0BA
:1020C00040E050E065E070E00E9442128091E8003C
:1020D0008E778093E8000895CF93DF93EC01909181
:1020E0001303943009F046C0809115018823D9F07C
:1020F000809116018823B9F09093E9008FEF9091B9
:10210000E800815095FD06C095E19A95F1F7000031
:102110008111F5CF8091E80085FF2CC040E050E0B0
:1021200060E170E017C081E08093E9008FEF90914B
:10213000E800815095FD06C095ED9A95F1F70000F5
:102140008111F5CF8091E80085FF14C040E050E098
:1021500068E070E0CE010E9442128091E8008E7724
:102160008093E80080E1FE01ACE7B2E001900D92BF
:102170008A95E1F7DF91CF91089580911203811143
:1021800009C00E94D7130E9434148091E200846039
:102190008093E2000895109212030895089508951F
:1021A0000C947B2242E061EC81E00E94511342E0FA
:1021B00061EC82E00E94511342E061EC83E00E94F6
:1021C000511342E161EC84E00C94511380911503AA
:1021D000833009F455C030F4813071F0823009F455
:1021E0008EC008958A3009F47AC08B3009F460C03B
:1021F000893009F09CC020C080911403813A09F015
:1022000096C08091E800877F8093E8008091180352
:1022100090911903892B21F460E18CE792E003C0CF
:1022200060E080E090E070E00E948D128091E80014
:102230008B778093E800089580911403813209F030
:1022400076C08091180390911903009719F00397B5
:1022500009F06DC08091E800877F8093E80080914D
:10226000E80082FD05C0809113038111F8CF5FC0A3
:102270008091F10080938C028091E8008B7753C0AD
:1022800080911403813A09F052C080911803909113
:102290001903892B09F04BC08091E800877F809358
:1022A000E8008091E80080FFFCCF8091150136C0E6
:1022B000809114038132D9F580911803909119030C
:1022C000892BA9F58091E800877F8093E8000E9420
:1022D000861380911603809315010C94BC1B80918A
:1022E0001403813221F58091E800877F8093E80014
:1022F0000E9486138091170380938D020895809128
:102300001403813AA1F48091E800877F8093E8006C
:102310008091E80080FFFCCF80918D028093F100D6
:102320008091E8008E778093E8000C9486130895DE
:1023300084B7877F84BF88E10FB6F89480936000EC
:10234000109260000FBE90E080E80FB6F894809382
:102350006100909361000FBE0E9429170E94D7135D
:102360000E9434148091E20084608093E2007894AB
:102370000E94BA160E942B178BE091E00E94D5169E
:1023800080911303853069F40E943C2280911103EF
:102390008823B1F30E946A22882391F30E942C12B1
:1023A000EFCF0E943317ECCF292F3327233031058D
:1023B000C9F064F42130310581F02230310509F093
:1023C00043C08DE690E028E433E042C0213231057D
:1023D000F1F02232310541F137C082E190E025EB86
:1023E00033E036C099278130910541F08230910564
:1023F00041F0892B49F5E4E4F3E005C0E6E1F3E0C0
:1024000002C0ECEEF2E0849190E09F0121C06430C4
:10241000D8F4E62FF0E0EE0FFF1FE255FE4F2081CB
:10242000318189E090E014C0643070F470E0FB0109
:10243000EE0FFF1FEA55FE4F20813181FB01EE5563
:10244000FE4F808190E004C080E090E020E030E02A
:10245000FA0131832083089580E189BD82E189BD3D
:1024600009B400FEFDCF8091D8008F7D8093D80005
:102470008091E00082608093E0008091E00081FD27
:10248000FCCF0895CF92DF92EF92FF920F931F93AC
:10249000CF93DF93EC018B016A010E94A513811198
:1024A00033C0C114D10439F0F60180819181081B39
:1024B000190BC80FD91FE12CF12C0115110519F1C9
:1024C0008091E80085FD16C08091E8008E778093AA
:1024D000E800C114D10449F0F60180819181E80E31
:1024E000F91EF182E08285E00FC00E94A5138823C7
:1024F00021F30AC089918093F10001501109FFEF87
:10250000EF1AFF0ADACF80E0DF91CF911F910F9190
:10251000FF90EF90DF90CF90089520911A033091B3
:102520001B032617370748F06115710539F4209110
:10253000E8002E772093E80001C0B90140E0611562
:102540007105A9F120911303222309F443C025301A
:1025500009F442C02091E80023FD40C02091E8002A
:1025600022FD32C02091E80020FFE9CF4091F30026
:102570002091F20030E0342BFC01CF016115710590
:1025800059F02830310540F481918093F100615079
:1025900071092F5F3F4FF1CF41E02830310509F03D
:1025A00040E02091E8002E772093E800C8CF411149
:1025B000C9CF0AC080911303882361F0853061F090
:1025C0008091E80083FD0AC08091E80082FFF2CF8D
:1025D00080E0089582E0089583E0089581E0089501
:1025E00020911A0330911B032617370748F0611515
:1025F000710539F42091E8002E772093E80001C09E
:10260000B901FC0120E06115710591F1809113037E
:10261000882309F440C0853009F43FC08091E80068
:1026200083FD3DC08091E80082FD2FC08091E800CD
:1026300080FFE9CF2091F3008091F20090E0922B8F
:102640006115710559F08830910540F4249120936B
:10265000F1003196615071090196F2CF21E008979F
:1026600009F020E08091E8008E778093E800CBCFDE
:102670002111CCCF0AC080911303882361F08530EB
:1026800061F08091E80083FD0AC08091E80082FF3C
:10269000F2CF80E0089582E0089583E0089581E01C
:1026A0000895982F973058F59093E900981739F0CE
:1026B0007091EC002091ED005091F00003C0242FA8
:1026C000762F50E021FF19C03091EB003E7F309310
:1026D000EB003091ED003D7F3093ED003091EB0049
:1026E00031603093EB007093EC002093ED00509339
:1026F000F0002091EE0027FF07C09F5FD3CF8F70BF
:102700008093E90081E0089580E0089580911403AA
:1027100087FF11C08091E80082FD05C080911303FE
:102720008111F8CF11C08091E8008B770BC08091A8
:102730001303882349F08091E80080FFF8CF80914F
:10274000E8008E778093E80008952091E4003091AE
:10275000E50095E64091EC00842F817040FF22C097
:102760008091E80080FD1CC080911303882391F0C4
:10277000853091F08091EB0085FD10C04091E40020
:102780005091E5004217530729F39A01915011F730
:1027900084E0089582E0089583E0089581E008953B
:1027A00080E008954091E80042FFDECF08950E9446
:1027B00045140E944D14E0EEF0E08081816080833A
:1027C000E8EDF0E080818F77808319BCA7EDB0E061
:1027D0008C918E7F8C9380818F7E808310921203E8
:1027E00008950F931F93CF93DF930E9445140E9487
:1027F0004D14C8EDD0E088818F7788838881806808
:10280000888388818F7D888319BC1092130310926E
:102810000F03109211031092100300EE10E0F80164
:1028200080818B7F808388818160888342E060E043
:1028300080E00E945113E1EEF0E080818E7F808382
:10284000E2EEF0E080818160808380818860808317
:10285000F80180818E7F8083888180618883DF9109
:10286000CF911F910F910895E8EDF0E080818F7E68
:102870008083E7EDF0E080818160808384E082BF27
:1028800081E0809312030C94F113E8EDF0E0808175
:102890008E7F80831092E20008951092DA001092E9
:1028A000E10008951F920F920FB60F9211242F93FB
:1028B0003F934F935F936F937F938F939F93AF93C8
:1028C000BF93EF93FF938091E10082FF0BC0809153
:1028D000E20082FF07C08091E1008B7F8093E100DE
:1028E0000E94B9168091DA0080FF1FC08091D80045
:1028F00080FF1BC08091DA008E7F8093DA00809188
:10290000D90080FF0DC080E189BD82E189BD09B495
:1029100000FEFDCF81E0809313030E94BD1005C02F
:1029200019BC109213030E94CB108091E10080FF2C
:1029300019C08091E20080FF15C08091E2008E7F77
:102940008093E2008091E20080618093E2008091B8
:10295000D80080628093D80019BC85E0809313036F
:102960000E94CF108091E10084FF30C08091E2008E
:1029700084FF2CC080E189BD82E189BD09B400FEDD
:10298000FDCF8091D8008F7D8093D8008091E100A9
:102990008F7E8093E1008091E2008F7E8093E20041
:1029A0008091E20081608093E20080910F03882390
:1029B00011F084E007C08091E30087FD02C081E050
:1029C00001C083E0809313030E94D0108091E10046
:1029D00083FF29C08091E20083FF25C08091E10040
:1029E000877F8093E10082E08093130310920F03AE
:1029F0008091E1008E7F8093E1008091E2008E7FE4
:102A00008093E2008091E20080618093E20042E0E6
:102A100060E080E00E9451138091F0008860809314
:102A2000F0000E94CE10FF91EF91BF91AF919F9166
:102A30008F917F916F915F914F913F912F910F9067
:102A40000FBE0F901F9018951F920F920FB60F9206
:102A500011242F933F934F935F936F937F938F93A3
:102A60009F93AF93BF93CF93DF93EF93FF93C09167
:102A7000E900CF708091EC00D82FD17080FDD0E8B4
:102A80001092E9008091F000877F8093F0007894A5
:102A90000E9468151092E9008091F0008860809390
:102AA000F000CD2BCF70C093E900FF91EF91DF9143
:102AB000CF91BF91AF919F918F917F916F915F91D6
:102AC0004F913F912F910F900FBE0F901F9018952F
:102AD0001F93CF93DF93CDB7DEB7AA970FB6F894C5
:102AE000DEBF0FBECDBFE4E1F3E088E08E0F909132
:102AF000F10091938E13FBCF0E94E6108091E800C5
:102B000083FF1FC18091140390911503492F50E05A
:102B10004A30510508F015C1FA01EA5AFF4F0C94EA
:102B2000752C803881F0823809F00BC18091180330
:102B30008F708093E9008091EB0085FB882780F9F6
:102B40001092E90006C08091100390911103911139
:102B500082609091E800977F9093E8008093F10065
:102B60001092F100C8C0282F2D7F09F0EAC08823F9
:102B700019F0823061F0E5C080911603813009F0D0
:102B8000E0C0933009F080E0809311032BC0809166
:102B90001603811127C0809118038F7009F4D1C0EA
:102BA0008093E9002091EB0020FF1CC0933021F4BA
:102BB0008091EB00806214C09091EB009061909343
:102BC000EB0021E030E0A90102C0440F551F8A95B7
:102BD000E2F74093EA001092EA008091EB008860EF
:102BE0008093EB001092E9008091E800877F86C017
:102BF0008111A7C0109116031F778091E3008078A0
:102C0000812B8093E3008091E800877F8093E80028
:102C10000E9486138091E80080FFFCCF8091E30042
:102C200080688093E300111102C082E001C083E05C
:102C30008093130386C08058823008F082C0809150
:102C40001603909117038C3D53E0950779F583E0C7
:102C50008A838AE289834FB7F894DE01139620E0D5
:102C60003EE051E2E32FF0E050935700E49120FF63
:102C700003C0E295EF703F5FEF708E2F90E0EA3077
:102C800010F0C79601C0C0968D939D932F5F24319D
:102C900049F74FBF8091E800877F8093E8006AE2A0
:102CA00070E0CE0101960E948D1214C0AE014F5FFC
:102CB0005F4F609118030E94D411BC01009709F482
:102CC00040C09091E800977F9093E80089819A81B5
:102CD0000E94F0128091E8008B778093E80031C069
:102CE000803879F58091E800877F8093E8008091B3
:102CF0000F038093F1008091E8008E778093E800C5
:102D00000E9486131EC081111CC090911603923040
:102D1000C0F48091E800877F8093E80090930F03D0
:102D20000E94861380910F03811106C08091E300F9
:102D300087FD02C081E001C084E0809313030E94FC
:102D4000D2108091E80083FF0AC08091E800877F5D
:102D50008093E8008091EB0080628093EB00AA965C
:102D60000FB6F894DEBF0FBECDBFDF91CF911F919C
:102D700008950895CF93809113038823A1F0C09103
:102D8000E900CF709091EC00892F817090FD80E870
:102D9000C82B1092E9008091E80083FD0E9468151D
:102DA000CF70C093E900CF910895909393028093E0
:102DB00092020895E0919202F0919302309721F0EF
:102DC0000190F081E02D099480E00895E091920255
:102DD000F0919302309721F00280F381E02D099465
:102DE0000895E0919202F0919302309721F00480CF
:102DF000F581E02D0994089520919002309191027F
:102E00008217930771F09093910280939002E09162
:102E10009202F0919302309721F00680F781E02D25
:102E20000994089520918E0230918F0282179307A2
:102E300071F090938F0280938E02E0919202F09154
:102E40009302309721F00084F185E02D09940895D4
:102E500008950C9428170E94AF220E9400090E9436
:102E600035230C94E4275F926F927F928F929F920A
:102E7000AF92BF92CF92DF92EF92FF920F931F9388
:102E8000CF93DF9300D000D01F92CDB7DEB70E9462
:102E900045099DE9C92E92E0D92E03E010E0AA244D
:102EA000A394B12C502E802F0E94C0094C01F60132
:102EB000729062906F016826792661147104A1F402
:102EC0000150110978F78FEF89838A831B820E9452
:102ED000B8228160782F9D838C8349815A816B81D0
:102EE0008D810E94E31738C08091F20281FD0E941B
:102EF000C9092BE030E07501022E02C0EE0CFF1C68
:102F00000A94E2F7C70186219721892B09F12983C9
:102F10005A828E209F2091E0892809F490E09B83BB
:102F20000E94B8228160782F9D838C8349815A81C9
:102F30006B818D810E94E317000F111FF801EB5682
:102F4000FD4F80819181E826F926F182E08204C05C
:102F50002150310980F6B4CF0E941C2510919402B3
:102F60000E94DA161817D1F00E94DA1680939402A4
:102F70000F900F900F900F900F90DF91CF911F91B6
:102F80000F91FF90EF90DF90CF90BF90AF909F9008
:102F90008F907F906F905F900C94EA080F900F9045
:102FA0000F900F900F90DF91CF911F910F91FF9095
:102FB000EF90DF90CF90BF90AF909F908F907F90D9
:102FC0006F905F900895CF93DF93CDB7DEB72B97C7
:102FD0000FB6F894DEBF0FBECDBF4F835887698709
:102FE0007A878B87DE01119686E0FD0111928A9522
:102FF000E9F785E0FE01379601900D928A95E1F799
:1030000049815A816B817C818D819E810E945A1EEB
:103010002B960FB6F894DEBF0FBECDBFDF91CF91D8
:103020000895CF93882309F4C2C0C82F823859F479
:103030000E94DA1681FDBBC089E30E9434210E9400
:10304000012289E30CC0833879F40E94DA1680FDEE
:10305000AEC083E50E9434210E94012283E50E94D4
:103060007621CF910C940122843859F40E94DA160B
:1030700082FD9DC087E40E9434210E94012287E4E2
:10308000EECF8CEF8C0F813A48F48C2F0E944C27A6
:1030900081118DC08C2F0E943421E3CF80E28C0FF0
:1030A000883048F4C77081E001C0880FCA95EAF7FC
:1030B0000E94BA21D6CF8BE58C0F833078F4C53AC5
:1030C00029F0C63A31F083E890E005C081E890E04D
:1030D00002C082E890E0CF910C94FC1688E58C0F3A
:1030E000833108F064C0C83A39F1C93A41F1CA3AAB
:1030F00049F1CB3A51F1CC3A59F1CD3A61F1C03BAB
:1031000069F1CE3A71F1CF3A79F1C13B81F1C23B1D
:1031100089F1C33B91F1C43B99F1C53BA1F1C63B99
:10312000A9F1C73BB1F1C83BB9F1C93BC1F1CA3BF9
:10313000C9F180E090E038C082EE90E035C089EEC1
:1031400090E032C08AEE90E02FC085EB90E02CC07A
:1031500086EB90E029C087EB90E026C08CEC90E0F5
:1031600023C08DEC90E020C083E891E01DC08AE888
:1031700091E01AC082E991E017C084E991E014C09F
:1031800081E292E011C083E292E00EC084E292E01C
:103190000BC085E292E008C086E292E005C087E2BB
:1031A00092E002C08AE292E0CF910C941217CF9184
:1031B0000895882309F44BC0823859F40E94DA1626
:1031C00081FF45C089E30E9434210E94012289E3E6
:1031D0000CC0833871F40E94DA1680FF38C083E592
:1031E0000E9434210E94012283E50E9476210C94E2
:1031F0000122843859F40E94DA1682FF28C087E43D
:103200000E9434210E94012287E4EFCF9CEF980FA7
:10321000913A58F390E2980F983050F4877091E00B
:1032200001C0990F8A95EAF7892F0E94C021DFCF4C
:103230009BE5980F933020F480E090E00C94FC160E
:10324000885A833120F480E090E00C94121708959E
:10325000882321F00E94BA210C940122089588232A
:1032600021F00E94C0210C94012208957F928F9238
:103270009F92AF92BF92CF92DF92EF92FF920F9305
:103280001F93CF93DF931F92CDB7DEB77C01C62E7D
:10329000772EFC01058102950F70128111110E9499
:1032A000D7210E942D21882379F0112369F080E233
:1032B0008C0D883048F082E00E9416210E942D215A
:1032C00091E0D82ED92601C0D12CE72DE295EF70E0
:1032D000F0E0E05AFF4F0C94752C872D807F072D6E
:1032E0000F70882311F00295007F112389F00023CD
:1032F00009F499C180E28C0D883020F4802F0E945F
:10330000BA2103C0802F0E94CA210E9401228BC1D2
:103310008C2D0E94D918002309F4C3C180E28C0DC2
:10332000883020F4802F0E94C02103C0802F0E948B
:10333000D0210E940122B5C1872D807F972D9F70DB
:10334000803211F4892F03C0892F8295807FCC2091
:1033500021F0F1E0CF16A1F01DC0112339F00023B8
:1033600019F1013009F50E94EA219BC1002319F0EF
:10337000013009F496C189830E94ED21898110C131
:10338000112321F0063008F08CC10EC0053008F082
:1033900088C106C1112359F0002331F0F70195814E
:1033A00090FF41C19F7095830E9428197AC1002324
:1033B00009F4F6C03EC1872D86958695837090E00E
:1033C000009719F0019761F06CC1112321F08C2D49
:1033D000972D937002C080E090E00E94FC1661C1BE
:1033E000112321F08C2D972D937002C080E090E086
:1033F0000E94121756C18C2D112319F00E9424240B
:1034000002C00E948C240E9411254BC1872D83701D
:1034100009F052C0111145C18C2D82958695877097
:10342000880F880F9C2D9F70892E912CA12CB12C78
:10343000082E04C0880C991CAA1CBB1C0A94D2F745
:10344000C4FE14C00FE010E020E030E0B901A80194
:1034500004C0440F551F661F771F8A95D2F7CB0112
:10346000BA01609570958095909503C060E070E01A
:10347000CB01272D26952695237030E0223031058B
:1034800069F02330310589F0682979298A299B2937
:103490002130310571F00E94A21F03C168297929EA
:1034A0008A299B290E94BE1FFCC00E94A21FC50141
:1034B000B4010E94861FF5C0112319F0872D817079
:1034C00001C08695882309F4ECC08C2D82958695E1
:1034D0008770880F880F9C2D9F70892E912CA12CAE
:1034E000B12C082E04C0880C991CAA1CBB1C0A9481
:1034F000D2F7C4FE14C00FE010E020E030E0B901C4
:10350000A80104C0440F551F661F771F8A95D2F784
:10351000CB01BA01609570958095909503C060E0ED
:1035200070E0CB01272D269526952370422F50E081
:103530004230510569F04330510589F068297929F5
:103540008A299B294130510571F00E947C20A9C035
:10355000682979298A299B290E949820A2C00E9463
:103560007C20C501B4010E9460209BC08C2D90E09E
:10357000FC01E05EF109E531F10508F050C0E059C9
:10358000FF4F0C94752C0C2D0F70872D8F7111230C
:1035900021F00E94F91F802F07CF0E941A20802F50
:1035A0000E942F197EC0112341F0053008F079C028
:1035B000872D8F710E943F2074C0063008F071C0C3
:1035C000F7CF112339F0872D8F710E94F91F69C041
:1035D0001123C9F3872D8F710E941A2062C0112315
:1035E00029F0872D8F710E94E41F5BC00E94DA1FB3
:1035F00058C0112351F0172D1F71812F0E94F91F00
:1036000063E0812F0E940D214CC081E00E941621B1
:10361000023008F446C082E00E94162142C0112305
:1036200031F0002381F28C2D0E9411183AC0002342
:1036300089F28C2D0E94D91834C0472D4F706C2D03
:10364000C7010E9455030E94FE1E2BC0111129C004
:10365000472D4F7050E042305105B9F04CF4411500
:10366000510581F041305105E1F40E940C2819C048
:103670004330510569F04430510599F48C2D0E9476
:103680005E280FC00E94F5270CC00E94282809C0A0
:103690000E943B2806C0472D4F706C2DC7010E9429
:1036A000CB05DD20F9F00E94092180FD1BC0F70148
:1036B00012820E9403210E94F91FC7010E94811BF0
:1036C0000E9403210F90DF91CF911F910F91FF90E6
:1036D000EF90DF90CF90BF90AF909F908F907F90B2
:1036E0000C941A200F90DF91CF911F910F91FF90B2
:1036F000EF90DF90CF90BF90AF909F908F907F9092
:1037000008950F931F93CF93DF93EC0188819981E4
:103710002B813C81232BB9F09F3F11F48F3F99F00F
:10372000CE010E94CA03882371F0688179818A8161
:103730000E94FF208C010E94B4200E947B1FB801D0
:10374000CE010E943619DF91CF911F910F910895FC
:103750000E94D7210E94E7210E94AC210E940122F1
:103760000E94C2250E94112580E090E00E94FC1674
:1037700080E090E00C9412170E94C7210C94A81BC3
:103780000E94F420292F22952F7030E02C30310533
:103790004CF42A3031056CF42250310922303105C5
:1037A000A8F407C02C30310569F02F30310551F0F5
:1037B0000DC0803F69F018F4803E40F409C0843F9A
:1037C00029F406C093FB882780F9089580E00895C6
:1037D00081E00895CF93DF9300D000D01F92CDB742
:1037E000DEB70F900F900F900F900F90DF91CF9159
:1037F0000895CF93DF9300D000D000D0CDB7DEB7CF
:1038000026960FB6F894DEBF0FBECDBFDF91CF91E5
:1038100008951F93CF93DF93C0919D0216E080918E
:103820009E02C81799F0D0E01C9FF0011D9FF00D7B
:103830001124E156FD4F4081518162817381848161
:1038400095810E94F91B2196C770E9CFDF91CF9136
:103850001F9108954091CF025091D0026091D10202
:103860007091D2028091D3029091D4020C94F91BF2
:103870008091D40282958F7009F054C08091D1025A
:10388000882309F44FC080919D02A0919E0260910F
:10389000CF027091D0024091D2025091D302B6E093
:1038A0008A1709F43FC090E041155105C1F17F3FEF
:1038B00011F46F3FA1F1B89FF001B99FF00D1124F1
:1038C000E156FD4F218172132AC02081621327C067
:1038D0002281211124C0238134812417350710F45B
:1038E00021503109241B350B283C3105C0F42091AF
:1038F000D4022F7020612093D40226E0289FF0018B
:10390000299FF00D1124EC55FD4F80818F7080614F
:1039100080838FEC92E00E94811B0C94091C01961D
:103920008770BECF0895CF92DF92EF92FF920F93F0
:103930001F93CF93DF93CDB7DEB762970FB6F8949E
:10394000DEBF0FBECDBF8C0185E0F801DE011D9604
:1039500001900D928A95E1F7D8014C9111965C91F6
:10396000119712966C9112971396CD90DC90149744
:103970003091CF027091D0028091D2029091D30207
:10398000009709F46BC17F3F19F43F3F09F466C10A
:10399000E090D102EE2009F4C0C02091D402C816F4
:1039A000D90628F0F601E81BF90BCF0104C0809579
:1039B00090958C0D9D1DFF24F394883C910578F023
:1039C000F12C207F09F0C6C07C2DD98AC88A89894C
:1039D0000E94EA1B8FEC92E00E94811BB1C0822FF3
:1039E000807F09F046C0751314C0341312C06111F2
:1039F00010C02F7020612093D4020E942A1C8FECEB
:103A000092E00E94811B8091D402D80115968C937C
:103A10002EC0CD2819F15F3F11F44F3FF9F0F62E7B
:103A200061111CC080919D0220919E0236E0821798
:103A300009F45AC090E0389FF001399FF00D11242D
:103A4000E156FD4F7181571306C07081471303C0C3
:103A50007281711103C001968770E9CFF62E66233B
:103A600009F418C18091D40281608093D402F12CB2
:103A700011C1751308C0341306C0611104C08091D0
:103A8000D402D801C3C04D875E878D859E856A8B21
:103A90000E94C01B6A898823E1F16623D1F120913D
:103AA000D402822F82958F7090E0029774F08091FB
:103AB000CF029091D00298878F831986DB86CA86C1
:103AC0002C87CE0107960E94811B86E0F801AFEC9F
:103AD000B2E001900D928A95E1F70E94381C0E9495
:103AE0002A1CFF24F394D6C04D875E878D859E8562
:103AF0000E94F420292F22952F7030E022303105CA
:103B00000CF0BCC09F7009F0B6C0805E883008F42D
:103B1000C1C0C8010E94811BE4CFC816D90608F4B1
:103B200053C0F601E81BF90BCF01883C910508F45E
:103B300050C0F12C7C2DD98AC88A89890E94EA1B41
:103B4000EFECF2E086E0DF011D928A95E9F70E9432
:103B50002A1CA0C0751314C0341312C0611110C008
:103B60008091D402F8018583C8010E94811B86E000
:103B7000EFECF2E0DF011D928A95E9F7FE2C8AC096
:103B80004D875E878D859E856A8B0E94C01B6A89E2
:103B9000882309F4BECF662309F4BBCF2091D40259
:103BA000822F82958F7090E002970CF48ECF8091D7
:103BB000CF029091D0029A8389831B82DD82CC82CE
:103BC0002E83CE0101967FCF809590958C0D9D1D03
:103BD000ACCFF62E662309F49CCF75132EC0341398
:103BE0002CC02091D40220FD1FC0822F82958F709F
:103BF000D9F0D80115962C9315978F3049F08F5F27
:103C0000982F9295907F822F8F70892B15968C9389
:103C1000C8010E94811B86E0F801AFECB2E0019080
:103C20000D928A95E1F793CF86E0F801AFECB2E010
:103C300001900D928A95E1F72DC04D875E878D85A5
:103C40009E850E94C01B811140CF8091D40281606B
:103C50008093D402C8010E94811B1CC0662309F412
:103C600058CF4D875E878D859E850E94C01B882317
:103C700009F44FCF2ACF811148CF0CC02430310531
:103C80000CF047CF9F7009F440CFF8019581907FE9
:103C900009F03BCF8F2D62960FB6F894DEBF0FBEB2
:103CA000CDBFDF91CF911F910F91FF90EF90DF90EB
:103CB000CF9008951F93CF93DF93CDB7DEB72C97A6
:103CC0000FB6F894DEBF0FBECDBF4F83588769870C
:103CD0007A878B879C87CE0107960E94931C882346
:103CE00069F08F8198852A853B85232BF1F19F3FD1
:103CF00009F063C08F3F09F060C037C086E0FE0165
:103D00003796DE01119601900D928A95E1F76F8149
:103D10007885EA85FB85309741F17F3F11F46F3F4D
:103D200021F120919E0230E0C90101968770992708
:103D300040919D0250E08417950709F447C06983BC
:103D40007A83FD83EC8396E0929FD001939FB00D20
:103D50001124A156BD4FFE01319601900D929A9506
:103D6000E1F780939E020E94091C16E080919D025B
:103D700090919E028917C1F1189FC00111248156AC
:103D80009D4F0E94931C882379F1E0919D021E9F14
:103D9000F0011124E156FD4F408151816281738110
:103DA000848195810E94F91B80919D0290E001968B
:103DB0008770992780939D02D9CF4F815885698557
:103DC0007A858B859C850E94F91BCFCF0E94BC1BF6
:103DD00010929E0210929D02EFECF2E086E0DF016D
:103DE0001D928A95E9F7C1CF2C960FB6F894DEBFE5
:103DF0000FBECDBFDF91CF911F910895EF92FF923B
:103E00000F931F93CF93DF938C01009709F46CC03D
:103E1000F12CEE24E394E8012196F8018491843793
:103E200040F4843008F051C0813081F0823019F1C3
:103E30005BC0853709F444C0A8F19CE7980F903720
:103E400008F052C08F770E94D91841C00E5F1F4FF3
:103E5000FE01C49180E28C0F883048F4C7708E2D2B
:103E600001C0880FCA95EAF70E94DA2114C08C2F8E
:103E70000E9411182DC00E5F1F4FFE01C49180E2F9
:103E80008C0F883058F4C7708E2D01C0880FCA95EA
:103E9000EAF70E94E0210E9401221AC08C2F0E94A2
:103EA000D91816C00E5F1F4FFE01C491CC2381F0BC
:103EB0008FE99FE00197F1F700C00000C150F6CFF5
:103EC0000E5F1F4FFE01F49003C00E9411188E0177
:103ED0008F2D882309F49FCFEFE9FFE03197F1F7A9
:103EE00000C000008150F5CFDF91CF911F910F915D
:103EF000FF90EF90089508956093D9027093DA02CD
:103F00008093DB029093DC020C94A81B0F931F9309
:103F10000091D9021091DA022091DB023091DC028B
:103F2000DC01CB01802B912BA22BB32B8093D902E8
:103F30009093DA02A093DB02B093DC021F910F9101
:103F40000C94A81B0F931F930091D9021091DA02D1
:103F50002091DB023091DC02DC01CB018023912334
:103F6000A223B3238093D9029093DA02A093DB02B9
:103F7000B093DC021F910F910C94A81B0F931F9319
:103F80000091D9021091DA022091DB023091DC021B
:103F9000DC01CB0180279127A227B3278093D90288
:103FA0009093DA02A093DB02B093DC021F910F9191
:103FB0000C94A81B1092D5021092D6021092D70230
:103FC0001092D8020C94A81B41E050E060E070E031
:103FD00004C0440F551F661F771F8A95D2F7409380
:103FE000D5025093D6026093D7027093D8020C94F6
:103FF000A81B41E050E060E070E004C0440F551F92
:10400000661F771F8A95D2F78091D5029091D602CC
:10401000A091D702B091D802482B592B6A2B7B2B49
:104020004093D5025093D6026093D7027093D80282
:104030000C94A81B41E050E060E070E004C0440F25
:10404000551F661F771F8A95D2F74095509560954A
:1040500070958091D5029091D602A091D702B0912F
:10406000D802482359236A237B234093D5025093D7
:10407000D6026093D7027093D8020C94A81B41E03B
:1040800050E060E070E004C0440F551F661F771FCA
:104090008A95D2F78091D5029091D602A091D7024D
:1040A000B091D802482759276A277B274093D50229
:1040B0005093D6026093D7027093D8020C94A81B39
:1040C0000F931F930091D5021091D6022091D70231
:1040D0003091D802DC01CB01802B912BA22BB32B8A
:1040E0008093D5029093D602A093D702B093D802C2
:1040F0001F910F910C94A81B0F931F930091D50251
:104100001091D6022091D7023091D802DC01CB0168
:1041100080239123A223B3238093D5029093D602C8
:10412000A093D702B093D8021F910F910C94A81BB3
:104130000F931F930091D5021091D6022091D702C0
:104140003091D802DC01CB0180279127A227B32729
:104150008093D5029093D602A093D702B093D80251
:104160001F910F910C94A81B0895CF92DF92EF92AC
:10417000FF920F931F93CF93DF938C01C090D902CE
:10418000D090DA02E090DB02F090DC028091D50260
:104190009091D602A091D702B091D802C82AD92A0C
:1041A000EA2AFB2ACFE1D0E0D701C6010C2E04C0D9
:1041B000B695A795979587950A94D2F780FF06C084
:1041C000B8018C2F0E945008019721F4219760F7C5
:1041D00080E001C08C2FDF91CF911F910F91FF9054
:1041E000EF90DF90CF900895CF93DF93EC010E9482
:1041F000B520BE010E945008DF91CF910895CB01F8
:104200000E94F42008958091DD028595859585951D
:1042100008958091DD028770089598E0899F90014C
:104220001124262B2093DD020C94F91F2091DD022E
:10423000809582238093DD02982F977069F430E097
:10424000482F552747FD50952417350729F08595A8
:10425000859585950C941A2008959091DD029770AC
:1042600081E009F480E0089590911501992321F0EF
:1042700090911601911109C02091170130911801F8
:10428000F90132969FEF40E01FC0982F96959695C2
:1042900096959F3050F5E0911701F0911801E90FC4
:1042A000F11D877021E030E0A90102C0440F551FC5
:1042B0008A95E2F7CA019181892B818308959F3FF6
:1042C00039F04F5F4E3041F051915813F8CF0DC087
:1042D0005111F7CF942FF5CF9F3F39F0F901E90F36
:1042E000F11D97FDFA958283089508959091150127
:1042F000992321F090911601911109C02091170185
:1043000030911801F9013296205F3F4F1FC0982F5E
:104310009695969596959F30F0F4E0911701F0915F
:104320001801E90FF11D877021E030E0A90102C0FA
:10433000440F551F8A95E2F7CA0180959181892320
:10434000818308953196E217F30729F0908198133D
:10435000F9CF1082F7CF089581E090E0E091170146
:10436000F0911801E80FF91F108201968031910534
:10437000A9F708959091F102892B8093F102089595
:1043800080959091F10289238093F1020895109213
:10439000F10208959091F002892B8093F002089524
:1043A00080959091F00289238093F00208951092F5
:1043B000F00208959091EF02892B8093EF02089507
:1043C00080959091EF0289238093EF0208951092D7
:1043D000EF0208958093DE0208951092DE020895A0
:1043E0008091170190911801FC0131969C01205F8A
:1043F0003F4F80E0919191118F5FE217F307D1F762
:104400000895E0911701F09118018091F1028083E5
:10441000E0911701F091180190818091F002892BB1
:104420008083E0911701F091180190818091EF0253
:10443000892B80838091DE02882361F0E09117014F
:10444000F09118019081892B80830E94F0218111C5
:104450001092DE0280911701909118010C94E616DB
:1044600020E0009739F0AC01415051098423952395
:104470002F5FF7CF822F089580911303843039F195
:104480001092F30220E488E190E00FB6F894A8952A
:10449000809360000FBE2093600080E00E94BC0209
:1044A00080E00E94EA0883B7817F846083BF83B77E
:1044B000816083BF7894889583B78E7F83BF88E1BE
:1044C0000FB6F89480936000109260000FBE0895BC
:1044D0000895089580E00E94BC020E9468220E9414
:1044E00045090E9469220E94CA0991E0811101C018
:1044F00090E0892F08950E94BC1B80E00E94BC02BE
:104500000E94E4270E94DA160C94EA081F920F9288
:104510000FB60F9211248F939F93AF93BF93809107
:10452000F302811113C08091F4029091F502A091E1
:10453000F602B091F7024196A11DB11D8093F402DD
:104540009093F502A093F602B093F702BF91AF915A
:104550009F918F910F900FBE0F901F90189582E042
:1045600084BD93E095BD9AEF97BD80936E0008954A
:104570002FB7F8948091F4029091F502A091F60281
:10458000B091F7022FBF0895CF92DF92EF92FF9282
:104590000F931F932FB7F8944091F4025091F502B6
:1045A0006091F6027091F7022FBF6A017B01EE2441
:1045B000FF248C0120E030E0C016D106E206F306AD
:1045C00010F4415051099A01281B390BC9011F9160
:1045D0000F91FF90EF90DF90CF9008951F920F9270
:1045E0000FB60F9211248F939F93AF93BF93809137
:1045F000F4029091F502A091F602B091F7020196B3
:10460000A11DB11D8093F4029093F502A093F602D0
:10461000B093F702BF91AF919F918F910F900FBE12
:104620000F901F9018950E94D713F8942FEF87EAE8
:1046300091E6215080409040E1F700C0000087E003
:1046400090EBDC0180931E0390931F03A093200343
:10465000B09321039CE088E10FB6F894A89580936D
:1046600060000FBE90936000FFCF0E947423811101
:1046700002C00E9450230E947F238093F2020E9476
:10468000872380931C0387FB882780F9809316017A
:104690000E948323682F70E080E090E00C947C1FE0
:1046A0006DEE7EEF80E090E00E949B2C60E082E067
:1046B00090E00E94892C60E083E090E00E94892CC9
:1046C00060E084E090E00E94892C60E085E090E06A
:1046D0000E94892C60E086E090E00E94892C6FEFB8
:1046E00087E090E00C94892C80E090E00E94832C7D
:1046F00021E08D3E9E4F09F020E0822F089582E058
:1047000090E00C947B2C83E090E00C947B2C84E074
:1047100090E00C947B2C682F84E090E00C94892C22
:1047200086E090E00C947B2C682F86E090E00C945F
:10473000892C87E090E00C947B2C682F87E090E038
:104740000C94892C8091FA0280FF0BC060911C01AF
:1047500085E0689FB00111247595679575956795FB
:104760002BC081FF09C060911C0185E0689FB001EA
:1047700011247595679520C082FF07C060911C01C8
:1047800085E0689FB001112417C09091FB02992326
:10479000D1F060911B01961788F720911C0185E0EC
:1047A000289F90011124929FA001939F500D1124E6
:1047B00070E0CA010E94612C6038710540F46115F7
:1047C000710539F002C065E070E0862F08958FE72B
:1047D000089581E008958091FA0280FF08C06091F9
:1047E0001A0170E0759567957595679521C081FFF1
:1047F00006C060911A0170E07595679519C082FF37
:1048000004C060911A0170E010C09091FB029923DE
:10481000C1F0609119019617A0F780911A01899F44
:10482000C001112470E00E94612C6038710528F4E9
:104830006115710521F0862F08958FE7089581E0B5
:10484000089561E070E0F4CF803F21F40E94A2233C
:10485000819504C0813F29F40E94A2238093FE0227
:104860000895823F21F40E94A223819504C0833FD2
:1048700029F40E94A2238093FD020895893F19F430
:104880000E94EB2305C08A3F31F40E94EB238195FF
:104890008093FF0208958B3F21F40E94EB238195C2
:1048A00004C08C3F29F40E94EB23809300030895F9
:1048B000843F21F48091FC02816017C0853F21F480
:1048C0008091FC02826011C0863F21F48091FC023D
:1048D00084600BC0873F21F48091FC02886005C092
:1048E000883F31F48091FC0280618093FC0208953E
:1048F0008D3F21F48091FA0281600BC08E3F21F43C
:104900008091FA02826005C08F3F29F48091FA02FB
:1049100084608093FA020895803F39F48091FE020A
:1049200087FF6CC01092FE0269C0813F29F480911C
:10493000FE021816BCF362C09091FD02823F29F47A
:1049400097FF5CC01092FD0259C0833F19F41916FD
:10495000CCF354C0893F41F48091FF0218160CF04B
:104960004DC01092FF024AC08A3F29F48091FF0295
:1049700087FF44C0F6CF8B3F39F48091000387FF57
:104980003DC0109200033AC08C3F29F4809100038F
:104990001816BCF333C0843F21F48091FC028E7F53
:1049A00017C0853F21F48091FC028D7F11C0863FA6
:1049B00021F48091FC028B7F0BC0873F21F4809112
:1049C000FC02877F05C0883F31F48091FC028F7E16
:1049D0008093FC0213C08D3F21F48091FA028E7FF8
:1049E0000BC08E3F21F48091FA028D7F05C08F3F6E
:1049F00029F48091FA028B7F8093FA028091FD0264
:104A000081110EC08091FE0281110AC08091FF02C7
:104A1000811106C080910003811102C01092FB0237
:104A200008958CEF92E00E94F1160E94B8229093B4
:104A3000F9028093F80208951F93CF93DF9380913A
:104A4000F8029091F9020E94C422AC019091FB02FD
:104A5000992321F020911D0130E006C020911E0114
:104A60008AE0289F900111244217530708F486C05A
:104A70008091FD02C091FE02D091FF0210910003CF
:104A8000811107C0C11176C0D11174C0111172C05B
:104A900075C09F3F19F09F5F9093FB02181624F496
:104AA0000E94A2238093FD028091FD0287FF05C032
:104AB0000E94A22381958093FD021C1624F40E947B
:104AC000A2238093FE028091FE0287FF05C00E9410
:104AD000A22381958093FE026091FD02662339F145
:104AE000C091FE02CC2319F1772767FD7095872FBF
:104AF000972F0E94832923E333E343E35FE30E947C
:104B0000932A0E9450296093FD026C2F772767FD3E
:104B10007095872F972F0E94832923E333E343E384
:104B20005FE30E94932A0E9450296093FE021D16A3
:104B300024F40E94EB238093FF028091FF0287FF01
:104B400005C00E94EB2381958093FF02111624F487
:104B50000E94EB23809300038091000387FF05C030
:104B60000E94EB23819580930003DF91CF911F91E9
:104B70000C9411259F3F09F08ECF96CFDF91CF91F6
:104B80001F910895ECEFF2E085E0DF011D928A9518
:104B9000E9F71092FB021092FA020895833081F136
:104BA00028F4813059F08230D1F00895853009F42D
:104BB00049C0B8F1863009F456C0089580911E01AD
:104BC000262F30E0280F311D2F3F310524F4680FC8
:104BD00060931E0108958FEF80931E0108958091C8
:104BE0001D01262F30E0280F311D2F3F310524F401
:104BF000680F60931D0108958FEF80931D01089544
:104C000080911C01262F30E0280F311D2F3F3105E8
:104C100024F4680F60931C0108958FEF80931C01AA
:104C2000089580911B01262F30E0280F311D2F3F62
:104C3000310524F4680F60931B0108958FEF809372
:104C40001B01089580911A01262F30E0280F311D95
:104C50002F3F310524F4680F60931A0108958FEFF8
:104C600080931A01089580911901262F30E0280FB2
:104C7000311D2F3F310524F4680F60931901089509
:104C80008FEF809319010895833011F128F481305A
:104C900049F0823091F00895853081F120F186301D
:104CA000C1F1089580911E01681720F4861B80933E
:104CB0001E01089510921E01089580911D0168172C
:104CC00020F4861B80931D01089510921D01089504
:104CD00080911C01681720F4861B80931C010895A5
:104CE00010921C01089580911B01681720F4861B07
:104CF00080931B01089510921B01089580911A0161
:104D0000681720F4861B80931A01089510921A01E7
:104D1000089580911901681720F4861B809319016A
:104D200008951092190108950F931F93873208F088
:104D300048C08E3108F08DC0803109F477C008F585
:104D4000873009F461C068F4863009F09DC0809115
:104D5000F202817F8E7F8093F20281E080930203D2
:104D600094C08B3009F489C08E3009F08DC08091D9
:104D7000F20282FB222720F991E0922790FB82F930
:104D80005EC0863109F479C060F4813109F07CC0DD
:104D90000E94BC1B9091160181E089278093160127
:104DA0006CC0893109F469C08B3109F06DC0809104
:104DB000F20281FB222720F991E0922790FB81F9F2
:104DC0003EC0883309F459C050F4893209F457C001
:104DD000853309F454C0873209F451C055C0833477
:104DE00009F44DC028F48A3308F44EC0895332C008
:104DF000883409F049C00E94BC1B0E94FA090E9435
:104E0000C1030E94132339C09091F202892F80952B
:104E1000817080FB90F929F0966098609093F2027F
:104E200034C0997F977F9093F20227C08091F2025D
:104E300083FB222720F991E0922790FB83F980934E
:104E4000F2029923D1F08091F20281608093F20204
:104E500014C08D5141E050E060E070E08A019B0198
:104E600004C0000F111F221F331F8A95D2F7C901FA
:104E7000B8010E947C1F0E94BC1B81E006C061E05B
:104E800070E080E090E0F5CF80E01F910F910895F1
:104E900080E0089580E00895CF93C82F80910203A9
:104EA000813069F018F08230C9F184C0E0911701B7
:104EB000F09118018081823209F07EC007C0E09134
:104EC0001701F09118018081823261F48C2F0E94C9
:104ED0004827811104C08C2F0E9494261DC081E0B8
:104EE00090E01AC08C2F0E944A27811114C0C4314F
:104EF00079F048F4CB3079F0C03109F061C082E03C
:104F00008093020308C0C93219F0C83321F058C099
:104F10001092020355C081E0817054C0C93291F1F2
:104F200020F5C43179F1B0F4C73009F047C08EE103
:104F300080931E0182E380931D018AE080931C010F
:104F400084E180931B0188E080931A0188E28093BA
:104F5000190134C0CE51C63088F5EC2FF0E0EA5488
:104F6000FE4F80818093010329C0CE34E9F020F404
:104F7000CB3421F56AE013C0C13579F0C235F1F4C4
:104F800061E00DC080910103882319F010920103A4
:104F900015C081E08093020315C061E006C08091D6
:104FA00001030E94CE250AC06AE0809101030E949D
:104FB000442604C01092020380E004C081E002C0D5
:104FC00080E0AACFCF9108950E947423811102C07E
:104FD0000E9450230E94902380931D0380FF02C0F3
:104FE000869501C080E00C94BC0280911D03982F2F
:104FF0009695292F30E0233031054CF49F5F990FAF
:105000008170892B816080931D030E94942380917D
:105010001D0386950C94BC0280911D03982F9695D4
:1050200091F09158990F8170892B80931D038E7F89
:1050300091E009F490E080911D0390FB80F980934A
:105040001D030E94942380911D0386950C94BC023D
:1050500080911D03982F909590FB80F980931D03FC
:105060000E94942380911D0380FF02C0869501C099
:1050700080E00C94BC0290911D03892F86958F5F70
:105080008F779170843028F4880F892B80931D03CB
:1050900002C090931D0380911D038E7F91E009F45F
:1050A00090E080911D0390FB80F980931D030E9486
:1050B000942380911D0386950C94BC0220911D03BE
:1050C000922F96958927982F990F822F8170892B7F
:1050D00080931D038E7F91E009F490E080911D0381
:1050E00090FB80F980931D030E94942380911D03FF
:1050F00086950C94BC0280911D03869508955058A6
:10510000BB27AA270ED0D1C1C2D130F0C7D120F021
:1051100031F49F3F11F41EF4B7C10EF4E095E7FBA4
:105120009FC1E92FD3D180F3BA17620773078407B1
:10513000950718F071F49EF5EBC10EF4E0950B2E77
:10514000BA2FA02D0B01B90190010C01CA01A001D9
:105150001124FF27591B99F0593F50F4503E68F134
:105160001A16F040A22F232F342F4427585FF3CF75
:10517000469537952795A795F0405395C9F77EF446
:105180001F16BA0B620B730B840BBAF09150A1F08F
:10519000FF0FBB1F661F771F881FC2F70EC0BA0F15
:1051A000621F731F841F48F4879577956795B7959D
:1051B000F7959E3F08F0B3CF9395880F08F0992795
:1051C000EE0F97958795089527D108F481E008950B
:1051D0000CD06BC163D140F05AD130F021F45F3F65
:1051E00019F03EC1511195C14FC170D198F3992367
:1051F000C9F35523B1F3951B550BBB27AA2762179B
:105200007307840738F09F5F5F4F220F331F441FDF
:10521000AA1FA9F333D00E2E3AF0E0E830D0915017
:105220005040E695001CCAF729D0FE2F27D0660F04
:10523000771F881FBB1F261737074807AB07B0E843
:1052400009F0BB0B802DBF01FF2793585F4F2AF059
:105250009E3F510568F004C15CC15F3FECF3983E8E
:10526000DCF3869577956795B795F7959F5FC9F7B6
:10527000880F911D9695879597F90895E1E0660F3F
:10528000771F881FBB1F621773078407BA0720F0B8
:10529000621B730B840BBA0BEE1F88F7E095089521
:1052A00004D06894B11135C1089518D188F09F5782
:1052B00090F0B92F9927B751A0F0D1F0660F771F62
:1052C000881F991F1AF0BA95C9F712C0B13081F042
:1052D0001FD1B1E008951CC1672F782F8827B85FD0
:1052E00039F0B93FCCF3869577956795B395D9F7A3
:1052F0003EF490958095709561957F4F8F4F9F4FAD
:105300000895E89409C097FB3EF4909580957095B8
:1053100061957F4F8F4F9F4F9923A9F0F92F96E901
:10532000BB279395F695879577956795B795F11176
:10533000F8CFFAF4BB0F11F460FF1BC06F5F7F4F13
:105340008F4F9F4F16C0882311F096E911C0772325
:1053500021F09EE8872F762F05C0662371F096E82E
:10536000862F70E060E02AF09A95660F771F881FFD
:10537000DAF7880F9695879597F9089588D018F0F1
:1053800011F08CD038F480C0C4C0E92F9FD0B0F3A6
:105390005523C9F3E7FB6217730784079507A8F144
:1053A00099F3E92FFF2788232AF03197660F771F9B
:1053B000881FDAF7952F5527442332F0915050403B
:1053C000220F331F441FD2F7BB27E91BF50B621BCB
:1053D000730B840BB109C1F222F4620F731F841F97
:1053E000B11D31972AF0660F771F881FBB1FEFCFC3
:1053F000915050405AF041F0882332F0660F771FE9
:10540000881F91505040C1F7939530C0869577958D
:1054100067959F5FD9F7F8CF990F0008550FAA0B32
:10542000E0E8FEEF16161706E807F907C0F01216B7
:105430001306E407F50798F0621B730B840B950BBA
:1054400039F40A2661F0232B242B252B21F408950F
:105450000A2609F4A140A6958FEF811D811D0895AC
:1054600097F99F6780E870E060E008959F3F31F012
:10547000915020F4879577956795B795880F911D82
:105480009695879597F908959FEF80EC08950024ED
:105490000A941616170618060906089500240A9499
:1054A00012161306140605060895092E0394000C1F
:1054B00011F4882352F0BB0F40F4BF2B11F460FFAE
:1054C00004C06F5F7F4F8F4F9F4F089557FD9058D7
:1054D000440F551F59F05F3F71F04795880F97FBB8
:1054E000991F61F09F3F79F0879508951216130672
:1054F0001406551FF2CF4695F1DF08C016161706A1
:105500001806991FF1CF86957105610508940895D5
:10551000E894BB2766277727CB0197F908957CDFAE
:1055200008F48FEF08950BD0C0CFB1DF28F0B6DFBD
:1055300018F0952309F094CFA7CF1124EACFC6DF46
:10554000A0F3959FD1F3950F50E0551F629FF00196
:10555000729FBB27F00DB11D639FAA27F00DB11DEF
:10556000AA1F649F6627B00DA11D661F829F222778
:10557000B00DA11D621F739FB00DA11D621F839FFF
:10558000A00D611D221F749F3327A00D611D231FD5
:10559000849F600D211D822F762F6A2F11249F5723
:1055A00050408AF0E1F088234AF0EE0FFF1FBB1F46
:1055B000661F771F881F91505040A9F79E3F5105E5
:1055C00070F04ECFA6CF5F3FECF3983EDCF38695AC
:1055D00077956795B795F795E7959F5FC1F7FE2B90
:1055E000880F911D9695879597F90895FA01EE0F0A
:1055F000FF1F30962105310599F16115710561F4A0
:105600008038BFE39B0749F168949038810561F0C9
:105610008038BFEF9B0741F0992342F5FF3FE1053A
:105620003105210511F1E8940894E795D901AA23E1
:1056300029F4AB2FBE2FF85FD0F310C0FF5F70F4DA
:10564000A695E0F7F73950F019F0FF3A38F49F7754
:105650009F930CD00F9007FC905808953EF014CF04
:1056600060E070E080E89FE308954FE79F775F93E5
:105670004F933F932F939ED02F913F914F915F91E6
:1056800052DF05C019F40EF0EBCE42CFFDCE26DF7F
:10569000C8F39638C0F707F80F92E8942BE33AEA7C
:1056A00048EB5FE74EDF0F920F920F924DB75EB758
:1056B0000F92C0D0EAE0F1E016D04F915F91EF91E8
:1056C000FF91E595EE1FFF1F49F0FE57E068442764
:1056D000EE0F441FFA95E1F74195550B32D00F902C
:1056E00007FE26C00895DF93CF931F930F93FF9279
:1056F000EF92DF927B018C01689405C0DA2EEF01F6
:105700001EDFFE01E894A5912591359145915591B3
:10571000AEF3EF0106DDFE019701A801DA9479F7F7
:10572000DF90EF90FF900F911F91CF91DF9108953F
:105730009B01AC0160E070E080E89FE349CD90CE32
:1057400095CECCDEE8F39923D9F3940F511DBBF32A
:105750009150504094F059F0882332F0660F771F33
:10576000881F91505040C1F79E3F510544F7880F64
:10577000911D9695879597F908955F3FACF0983EF7
:105780009CF0BB27869577956795B79508F4B1602F
:105790009395C1F7BB0F58F711F460FFE8CF6F5F27
:1057A0007F4F8F4F9F4FE3CFB4CE0EF05FCE6CCEC6
:1057B000689456CE93DEC8F39923D1F3C6F3DF93F2
:1057C000CF931F930F93FF92C92FDD2788232AF0D1
:1057D0002197660F771F881FDAF720E030E040E856
:1057E0005FEB9FE3883920F0803E30F021968F7781
:1057F00087DCE2E3F1E003C083DCEFE5F1E073DF97
:105800008B01BE01EC01FB2E6F5771097595771F57
:10581000880B990B78DD28E132E741E35FE38FDE07
:10582000AF2D9801AE01FF900F911F91CF91DF91A5
:1058300078DC3BCEFA01DC01AA0FBB1F9B01AC0157
:10584000BF5728F422273327442750781FC0B75169
:1058500088F4AB2F0024469537952795011CA39516
:10586000D2F3002069F0220F331F441FB395DAF3FF
:105870000DD045CC61307105A0E88A07B94630F4F7
:105880009B01AC016627772788279078309621F016
:1058900020833183428353830895AA1BBB1B51E1AC
:1058A00007C0AA1FBB1FA617B70710F0A61BB70B90
:1058B000881F991F5A95A9F780959095BC01CD0135
:1058C000089597FB072E16F4009407D077FD09D0B2
:1058D0000E944D2C07FC05D03EF4909581959F4F7A
:1058E0000895709561957F4F0895EE0FFF1F059005
:1058F000F491E02D0994F999FECF92BD81BDF89AFB
:10590000992780B50895A8E1B0E042E050E00C94FA
:10591000A32C262FF999FECF92BD81BDF89A01974D
:1059200000B4021639F01FBA20BD0FB6F894FA9AE7
:10593000F99A0FBE08950196272F0E948A2C0C9485
:10594000892CDC01CB01FC01F999FECF06C0F2BD28
:10595000E1BDF89A319600B40D9241505040B8F72D
:065960000895F894FFCF4A
:10596600640007000CFF0000003F64DE0F6C104966
:10597600101510E10F0101DF022808140A321E007B
:1059860002040507090B0C0E1011131517181A1C23
:105996001D1F2123242628292B2D2F30323435375D
:1059A600393B1F0F03764F5F6F7F4969437909596A
:1059B60053633149803F5D8B803FF8BF803FCAE12A
:1059C600803F73ED803FCAE1803FF8BF803F5D8B2B
:1059D600803F3149803F0000803FF16D7F3F75EA8F
:1059E6007E3F4C827E3F833F7E3F84287E3F833FBF
:1059F6007E3F4C827E3F75EA7E3FF16D7F3F000021
:105A0600803F3F4D3639830436040004C7035A03EA
:105A160073038C03A50301020304050607080900A6
:00000001FF
